:040000008231142A0B
:100008007E1480312100901E0A280B28122A200015
:10001800901E0F281028122A953140258031200083
:100028006B082100C700003020000E190130EB00DA
:100038006B08031D202821282928210047080319B7
:10004800262827282928B901B90A20006D08210087
:10005800C900003020000C180130ED006D08031DA8
:10006800362837284E282100490803193C283D28FE
:1000780041282000CF01CF0A50280130FC007C081D
:10008800B80706303802031C4A284B28502820009D
:10009800CF01CF0A2100B80120006C082100C80058
:1000A800003020008C180130EC006C08031D5D281E
:1000B8005E287528210048080319632864286828E1
:1000C8002000CE01CE0A77280130FC007C08B70753
:1000D80006303702031C7128722877282000CE01C9
:1000E800CE0A2100B70120004608470403197D28DD
:1000F8007E2882280130C6020030C73B4508803A76
:10010800FC0080307C02031D8B2801304402031C54
:100118008E288F289428FF302000C407FF30C53D63
:1001280021003208330403199A289B28412920000A
:10013800CD01CD0A2100A801A90120004308F10042
:100148004208F0000530F2000030F30096314426F2
:1001580080317108F7007008F60095315325803119
:10016800FD0132307D02031CBA28BB28BC28DF28D9
:1001780005309531C125803171082000B90070081B
:10018800B800390821002902031DCE2820003808AC
:10019800210028020318D128D228DA28200039089B
:1001A8002100A900200038082100A8000130FC0027
:1001B8007C08FD07B528210028082000A0002100A0
:1001C80029082000A100A201A3010030F30000309B
:1001D800F2000030F1002830F0002308F700220870
:1001E800F6002108F5002008F400883192208031BB
:1001F80073082000A3007208A2007108A10070080B
:10020800A0004008F0004108F100890D893B8909E8
:10021800F200F3002308F7002208F6002108F50091
:100228002008F40088319220803173082000A30050
:100238007208A2007108A1007008A0000B30A33654
:10024800A20CA10CA00C890B23292108B9002008B5
:10025800B80039083F02031D332938083E02031845
:10026800362937293B293908BF003808BE00013034
:100278002100B2020030B33BD22920004D080319F7
:1002880046294729D2292100B001B101FD013230A8
:100298007D02031C502951295229752905309531B1
:1002A800C125803171082000B9007008B8003908EC
:1002B80021003102031D6429200038082100300282
:1002C8000318672968297029200039082100B1001E
:1002D800200038082100B0000130FC007C08FD0730
:1002E8004B292000CD010030F600F7009531532549
:1002F8008031210030082000A000210031082000B2
:10030800A100A201A3010030F3000030F200003088
:10031800F1002830F0002308F7002208F600210831
:10032800F5002008F40088319220803173082000FD
:10033800A3007208A2007108A1007008A00040087C
:10034800F0004108F100890D893B8909F200F300AA
:100358002308F7002208F6002108F5002008F40019
:1003680088319220803173082000A3007208A2000F
:100378007108A1007008A0000B30A336A20CA10CD4
:10038800A00C890BC1292108B9002008B800390838
:100398002100AF00200038082100AE0020003C08F2
:1003A8003D040319D829D929F02901302100AC07C7
:1003B8000030AD3D00302D02143003192C02031C0F
:1003C800E629E729F029AC01AD012000CC01CC0ACF
:1003D8000130BC020030BD3B01302100AA070030CB
:1003E800AB3D00302B02143003192A02031CFD29EF
:1003F800FE29122AAA01AB0120003A083B0403197E
:10040800062A072A0B2A0130BA020030BB3B4B08E8
:1004180003190F2A102A122A0130CB027E10090074
:100428008231162A90308400943085006B30860023
:10043800003087000330883100208231A5308400E5
:1004480094308500C330860000308700073088313B
:1004580000208231FD0120308400003085003030DA
:1004680094319F248231A0308400003085002330ED
:1004780094319F2482317E1020008231432A8631B4
:10048800B026823164002100390803194C2A4D2A0C
:10049800C72AB9012000CF01CE01BC01BD01C601A8
:1004A800C701FF30C400FF30C5000A30CB004A083E
:1004B800803A7F3E031C612A622A672A0130E900DC
:1004C8006908CA076D2ACA1F6A2A6B2A6D2ACA01D7
:1004D800CA0A4A08803A703E031C732A742AC72A3B
:1004E8008531382582312000CA01CA0AC72A8F31CE
:1004F8007D2782310F2B8C31262482310F2B8931B5
:10050800A22182310F2B8C31BB2482310F2B8B31EE
:10051800DF2382310F2B8B31982382310F2B8931C6
:100528002C2182310F2B8931672182310F2B8931A0
:10053800DD2182310F2B8A31552282310F2B8A31EE
:10054800D22282310F2B8D31C02582310F2B85317C
:10055800FD2582310F2B8A31932282310F2B963160
:10056800862682310F2B97316E2782310F2B8831E7
:10057800C52082310F2B88312F2082310F2B8631F5
:10058800B02682310F2B20004A08E900EA01E91B56
:10059800EA036A08003A0319D52AFF3A0319042B1B
:1005A800C32A6908013A03197B2A033A03197F2AE7
:1005B800013A0319832A073A0319872A013A0319CA
:1005C8008B2A033A03198F2A013A0319932A0F3AFF
:1005D8000319972A013A03199B2A033A03199F2AF8
:1005E800013A0319A32A073A0319A72A013A03195A
:1005F800AB2A033A0319AF2A013A0319B32AC32ACB
:100608006908FD3A0319BF2A033A0319BB2A013ABC
:100618000319B72AC32A2000460847040319152BD3
:10062800162B192B22000C111B2B22000C15200055
:100638004508803AE90080306902031D252B013006
:100648004402031C282B292B2C2B22000E102E2BA6
:1006580022000E1420004B080319332B342B372BA0
:1006680022000E12392B22000E1621004408200009
:100678003B06031D432B2100430820003A060319BB
:10068800462B472B792B3B082100C40020003A0851
:100698002100C30020003A083B04031D542B552BAE
:1006A800792B8E312726823120005D08B7005C083F
:1006B800B6005830BA000230BB0029083702031DC3
:1006C800672B2808360203186A2B6B2B6F2BFE301A
:1006D800CA00C801C80A0E1F722B732B762B210083
:1006E800B601792B2100B601B60A20004A0849064E
:1006F80003197F2B802B842BCF01CE014A08C90018
:10070800FA300032890B852B462A8231142A2000C0
:100718004F080319902B912BFB2BCF010A30CB00EC
:1007280000305D020A3003195C0203189C2B9D2BD4
:10073800A22B0130E2000030E300C22B00305D0242
:10074800643003195C020318AA2BAB2BB02B0A30B8
:10075800E2000030E300C22B27305D02103003199D
:100768005C020318B82BB92BBE2B6430E2000030B2
:10077800E300C22BE830E2000330E30062085C07C4
:10078800E00063085D3DE1006308D1006208D00025
:100798006108D3006008D2008A3118228331200012
:1007A8005108E1005008E0006308D1006208D00059
:1007B8006108D3006008D2008731DE27833120002A
:1007C8005108E1005008E00061085B02031DEE2BB0
:1007D80060085A020318F12BF22BF62B5B08E10094
:1007E8005A08E0006108D9006008D800712C4E084A
:1007F8000319FF2B002C6D2CCE010A30CB000030E2
:100808005D020B3003195C0203180B2C0C2C112C05
:100818000130E2000030E300312C00305D02653029
:1008280003195C020318192C1A2C1F2C0A30E20039
:100838000030E300312C27305D02113003195C02CF
:100848000318272C282C2D2C6430E2000030E300FC
:10085800312CE830E2000330E30062085807DE007C
:100868006308593DDF005F085D02031D3D2C5E08EB
:100878005C02031C402C412C682C62085C02E000DE
:1008880063085D3BE1006308D1006208D00061089D
:10089800D3006008D2008A31182283312000510821
:1008A800E1005008E0006308D1006208D000610848
:1008B800D3006008D2008731DE2783312000510839
:1008C800E1005008E000F62B5908E1005808E00064
:1008D800F62B5D08D9005C08D8000800003020001D
:1008E800D800F030D9000030D200F030D300973172
:1008F80015278431200053082100A3002000520846
:100908002100A20002302000D8070030D93D590844
:10091800D3005808D2009731152784312000530896
:10092800B3005208B2000230D8070030D93D590848
:10093800D3005808D2009731152784312000530876
:10094800B1005208B0000230D8070030D93D59082C
:10095800D3005808D2009731152784312000530856
:10096800AF005208AE000230D8070030D93D590810
:10097800D3005808D2009731152784312000530836
:10098800AD005208AC000230D8070030D93D5908F4
:10099800D3005808D2009731152784312000530816
:1009A800AB005208AA000230D8070030D93D5908D8
:1009B800D3005808D20097311527843120005308F6
:1009C800A9005208A8000230D8070030D93D5908BC
:1009D800D3005808D20097311527843120005308D6
:1009E800A7005208A6000230D8070030D93D5908A0
:1009F800D3005808D20097311527843120005308B6
:100A0800A5005208A4000230D8070030D93D590883
:100A1800D3005808D2009731152784312000530895
:100A2800B5005208B4000230D8070030D93D590843
:100A3800D3005808D2009731152784312000530875
:100A4800C1005208C0000230D8070030D93D59080B
:100A5800D3005808D2009731152784312000530855
:100A6800C3005208C200080000302000DC00F0304B
:100A7800DD000030D800F030D90021002308200024
:100A8800DB00210022082000DA00883106208531A9
:100A980002302000DC070030DD3D5D08D9005C082D
:100AA800D8003308DB003208DA00883106208531A7
:100AB80002302000DC070030DD3D5D08D9005C080D
:100AC800D8003108DB003008DA008831062085318B
:100AD80002302000DC070030DD3D5D08D9005C08ED
:100AE800D8002F08DB002E08DA008831062085316F
:100AF80002302000DC070030DD3D5D08D9005C08CD
:100B0800D8002D08DB002C08DA0088310620853152
:100B180002302000DC070030DD3D5D08D9005C08AC
:100B2800D8002B08DB002A08DA0088310620853136
:100B380002302000DC070030DD3D5D08D9005C088C
:100B4800D8002908DB002808DA008831062085311A
:100B580002302000DC070030DD3D5D08D9005C086C
:100B6800D8002708DB002608DA00883106208531FE
:100B780002302000DC070030DD3D5D08D9005C084C
:100B8800D8002508DB002408DA00883106208531E2
:100B980002302000DC070030DD3D5D08D9005C082C
:100BA800D8003508DB003408DA00883106208531A2
:100BB80002302000DC070030DD3D5D08D9005C080C
:100BC800D8004108DB004008DA008831062085316A
:100BD80002302000DC070030DD3D5D08D9005C08EC
:100BE800D8004308DB004208DA0088310620853146
:100BF8000800200049084A060319032E042E262E51
:100C0800D430D7009830D80095311325853120008D
:100C18004008003ED900F830413DDA00BA308F3143
:100C280004278531BD3096316326853121002F0890
:100C38002000E60021002E082000E5008B31552316
:100C48008531AF2E0030D0000430D1000030D20002
:100C58000C30D3004108D5004008D4008C317024F2
:100C6800853120005108B9005008B80039084106FC
:100C7800031D402E380840060319432E442EAF2E7C
:100C88003908C1003808C000D430D7009830D800DF
:100C980095311325853120004008003ED900F830F1
:100CA800413DDA00BA308F3104278531BD309631A5
:100CB80063268531210030082000A000210031087A
:100CC8002000A100A201A3010030D3000030D2000F
:100CD8000030D1002830D0002308D7002208D600E1
:100CE8002108D5002008D4008831F820853120005B
:100CF8005308A3005208A2005108A1005008A00000
:100D08004008D0004108D100890D893B8909D200EB
:100D1800D3002308D7002208D6002108D5002008D0
:100D2800D4008831F820853120005308A3005208E8
:100D3800A2005108A1005008A0000B30A336A20C55
:100D4800A10CA00C890BA22E2108E6002008E500C2
:100D58008B3155238531080096310B2686318B312E
:100D6800132386318B170B17843172248631553043
:100D780021002206AA30031923060319C42EC52E02
:100D8800F92E5530A200AA30A3002C302000B20062
:100D98000130B3006430B0000030B1003230AE0032
:100DA8000030AF005830AC000230AD000A30AA0065
:100DB8000030AB002030A8001C30A900A830A600E5
:100DC8006130A700A030A4000F30A5000030B400A7
:100DD8000830B5000030C0000830C1006430C200DF
:100DE8000030C30085313825863105302000BC002D
:100DF8000030BD000930D7009830D8009531132550
:100E08008631182F4C0803190A2F0B2F182FCC01E5
:100E18003D08DA003C08D900BA308F310427863102
:100E2800BA309431F924863120003C083D04031D72
:100E38001E2F1F2F062FCF01CE012100B901200040
:100E4800CA01CA0AC901C601C701FF30C400FF3080
:100E5800C500BC01BD012100B201B3010A30200068
:100E6800CB000E1F382F392F3C2F2100B6013F2F02
:100E78002100B601B60A8E312726863120005D088A
:100E8800B7005C08B6000800E0302000D7009830B2
:100E9800D80095311325873132302100CA07003038
:100EA800CB3D64302000D0000030D10021004B0839
:100EB8002000D30021004A082000D2008A311822DD
:100EC8008731200051082100CB0020005008210064
:100ED800CA004A084B04031D722F732F7C2FC4309D
:100EE8002000D3009830D4009531D82587319A2F27
:100EF8004B082000DA0021004A082000D900BA3047
:100F08008F310427873121003F08BE004008BF0009
:100F18002E30C000BE30963163268731C83020009D
:100F2800D3009830D4009531D8258731CA302000B5
:100F3800D7009830D80095312225873132302100EA
:100F4800CC070030CD3D64302000D0000030D10007
:100F580021004D082000D30021004C082000D200B9
:100F68008A3118228731200051082100CD00200045
:100F780050082100CC004D082000DA0021004C0860
:100F88002000D900BA308F310427873121003F086B
:100F9800BE004008BF002E30C000BE309631632628
:100FA8008731C8302000D3009830D4009531D82537
:100FB800873108002000D401D501501CE42FE52F0B
:100FC800E92F5208D4075308D53D0130D235D30D47
:100FD800890BEA2F0130D136D00C890BEF2F50083E
:100FE8005104031DF82FF92FE12F5508D10054089B
:060FF800D0000800080013
:10100000FE0012001E00FE0B0128003420005908CB
:10101000D3005808D20097311527883120005B088B
:101020005306031D15285A085206031918281928B3
:101030002E285908D1005808D0005B08D2009631FC
:10104000F126883120005808013ED0000030593D7B
:10105000D1005A08D2009631F126883108002000CC
:1010600036083704031D352836283C2849084A0627
:1010700003193B283C284E286C30D7009830D80004
:1010800095311325883121002F082000E60021002A
:101090002E082000E5008B315523883122000C11E9
:1010A000FA300032890B512822000C15A1302000A3
:1010B000E700B530890B5A28E70B5A2800320800A0
:1010C000210021082000DA00210020082000D9009A
:1010D000BA308F3104278831C030953106258831E8
:1010E000BD302000D3009830D4009531D825883108
:1010F00021002108C6002008C5002000360837045A
:10110000031D832884288A284A0849060319892848
:101110008A2891283708E6003608E50097319E278F
:10112000883108000030FB000030FA000030F90080
:101130000030F800701C9D289E28A6287408F80727
:101140007508F93D7608FA3D7708FB3D0130F43526
:10115000F50DF60DF70D890BA7280130F336F20CCB
:10116000F10CF00C890BAE28730872047104700442
:10117000031DBB28BC289A287B08F3007A08F200DC
:101180007908F1007808F0000800200049084A06B4
:10119000031DCB28CC28D12848080319D028D128F2
:1011A000E128C801AB30D7009830D800953113251D
:1011B000883120003708E6003608E50097319E2781
:1011C000883122000E10FA300032890BE428220008
:1011D0000E1402302000E800E630E7006030890B92
:1011E000EF28E70BEF28E80BEF280000E1280800C4
:1011F00000302000DB000030DA000030D900003081
:10120000D800501C042905290D295408D807550871
:10121000D93D5608DA3D5708DB3D0130D435D50DB0
:10122000D60DD70D890B0E290130D336D20CD10C37
:10123000D00C890B15295308520451045004031D86
:101240002229232901295B08D3005A08D200590812
:10125000D1005808D0000800200049084A060319A8
:101260003229332943299030D7009830D80095315E
:101270001325893120002D08E6002C08E500953162
:101280007F25893166290530D8000030D90010301B
:10129000DA002730DB002D08DD002C08DC0083316C
:1012A0008B23893120005908B9005808B8002D084F
:1012B0003906031D5D292C083806031960296129A8
:1012C00066293908AD003808AC003A29080020002A
:1012D00049084A0603196D296E297E299930D700DD
:1012E0009830D80095311325893120002B08E6006D
:1012F0002A08E50095317F258931A1290530D800DC
:101300000030D900E830DA000330DB002B08DD00C4
:101310002A08DC0083318B23893120005908B90069
:101320005808B8002B083906031D98292A083806E2
:1013300003199B299C29A1293908AB003808AA0068
:1013400075290800200049084A060319A829A92977
:10135000B9295A30D7009830D800953113258931F2
:1013600020004308E6004208E500953195258931C3
:10137000DC293230D0000030D1006430D20000309F
:10138000D3004308D5004208D4008C317024893141
:1013900020005108B9005008B80043083906031D61
:1013A000D329420838060319D629D729DC29390858
:1013B000C3003808C200B0290800200049084A06C6
:1013C0000319E329E429F4293F30D7009830D800E5
:1013D00095311325893120002908E6002808E50009
:1013E00097319E278931172A7030D8001730D900DD
:1013F000E830DA001C30DB002908DD002808DC00BA
:1014000083318B23893120005908B9005808B8006E
:1014100029083906031D0E2A280838060319112A3F
:10142000122A172A3908A9003808A800EB29080051
:101430002000D601D701500851040319202A212A7F
:10144000502AD501D50A2D2A0130D035D10D890B6E
:10145000252A0130D4005408D507D11F302A312A5B
:10146000242A0130D635D70D890B322A5108530270
:10147000031D3C2A50085202031C3F2A402A452AD9
:101480005008D2025108D33B56140130D136D00C4B
:10149000890B462A0130D502031D4F2A502A312AD2
:1014A0005708D1005608D0000800200049084A0615
:1014B00003195B2A5C2A6F2A3F082100CB00200019
:1014C0003E082100CA00200027082100CD0020008E
:1014D00026082100CC00873148278A31922AE8303B
:1014E000D8000330D900B830DA008830DB00270894
:1014F000DD002608DC0083318B238A312000590867
:10150000B9005808B80027083906031D892A26089B
:10151000380603198C2A8D2A922A3908A700380820
:10152000A6005C2A0800200049084A060319992AE7
:101530009A2AA92A1230D7009830D800953113255D
:101540008A3124302000D7009830D80095312225E8
:101550008A3120008E1CAD2AAE2AB22A0530C60080
:101560000030C7000D1FB52AB62ABA2A0530C400BC
:101570000030C500460847040319BF2AC02AC32A01
:1015800022000C11C52A22000C1520004408450435
:101590000319CB2ACC2ACF2A22000E10D12A2200EE
:1015A0000E140800200049084A060319D82AD92A2F
:1015B000E92A6330D7009830D800953113258A3155
:1015C00020002508E6002408E5008B3155238A31E8
:1015D000122B0030D800D9001030DA002730DB00A1
:1015E0002508DD002408DC0083318B238A312000AC
:1015F0005908B9005808B80025083906031D022B00
:10160000240838060319052B062B122B3908A500D0
:101610003808A4006330D7009830D80095311325DE
:101620008A31E02A0800943193248B31073020005E
:10163000D3007D30890B1A2BD30B1A2B38309631FF
:10164000A9268B3139309631A9268B311430963149
:10165000A9268B3176309631A9268B3150309631C0
:10166000A9268B316C309631A9268B3104302000AD
:10167000D3003D30890B3A2BD30B3A2B0032383054
:101680009631A9268B310C309631A9268B31013049
:101690009631A9268B3111302000D3003A30890BC6
:1016A0004F2BD30B4F2B0000080020006508660469
:1016B00003195B2B5C2B902B0530E5070030E63DD2
:1016C0000A30D0000030D1006608D3006508D2008F
:1016D0008A3118228B3120005108E6005008E500BD
:1016E0006608DA006508D900BA308F3104278B31DB
:1016F00021003C08BB003D08BC003E08BD003F087F
:10170000BE002E30BF00BB309431F9248B31C8307D
:101710002000D3009830D4009531D8258B31972BF9
:101720004830D7009830D800953122258B310800F9
:10173000200049084A0603199E2B9F2BBB2BA23081
:10174000D7009830D800953113258B310A3020000E
:10175000D0000030D1002F08D3002E08D2008A31EB
:1017600018228B3120005108E6005008E500953121
:101770007F258B31DE2B0A30D8000030D900323083
:10178000DA000030DB002F08DD002E08DC0083319A
:101790008B238B3120005908B9005808B8002F0856
:1017A0003906031DD52B2E0838060319D82BD92B43
:1017B000DE2B3908AF003808AE00A62B0800200049
:1017C00049084A060319E52BE62B022C2D30D700D9
:1017D0009830D800953113258B310A302000D00085
:1017E0000030D1003108D3003008D2008A311822ED
:1017F0008B3120005108E6005008E50095317F2527
:101800008B31252C0A30D8000030D900B830DA00EE
:101810000B30DB003108DD003008DC0083318B2326
:101820008B3120005908B9005808B8003108390632
:10183000031D1C2C3008380603191F2C202C252CC6
:101840003908B1003808B000ED2B08002000490825
:101850004A06031D2C2C2D2C322C48080319312C40
:10186000322C462CC8017E30D7009830D8009531F4
:1018700013258C3120003308E6003208E50095314D
:10188000AB258C312000BC01BD016F2C6430D80029
:101890000030D900B830DA000B30DB003308DD004F
:1018A0003208DC0083318B238C3120005908B900C9
:1018B0005808B80033083906031D602C3208380672
:1018C0000319632C642C6F2C3908B3003808B2005C
:1018D0003308E6003208E5009531AB258C3108006D
:1018E00020004F080319752C762C922CCF010A305A
:1018F000CB005408013ED8000030553DD9005908AE
:101900005302031D852C580852020318882C892C79
:101910008D2C5308D9005208D8005908D100580816
:10192000D000BA2C4E080319962C972CB62CCE0159
:101930000A30CB005008013ED6000030513DD700A0
:1019400057085502031DA62C56085402031CA92C47
:10195000AA2CB12C5408FF3ED800FF30553DD900C9
:101960008D2C5108D9005008D8008D2C5508D10075
:101970005408D0000800200049084A060319C12C69
:10198000C22CD12C5130D7009830D8009531132576
:101990008C3120003308E6003208E5009531AB2594
:1019A0008C3101302000D8000030D9000330DA003B
:1019B0000030DB000230DC000030DD0083318B239F
:1019C0008C3120005908B9005808B8000330380697
:1019D0003904031DEC2CED2C012D8E3193268C3116
:1019E00051302000D7009830D800953113258C3124
:1019F00020003308E6003208E5009531AB258C3134
:101A00000B2D38033904031D062D072D0B2D023035
:101A1000CA00C801C80A08002000D601D31F112D32
:101A2000122D192DD209D309D20A0319D30AD601CE
:101A3000D60AD11F1C2D1D2D222DD009D109D00A67
:101A40000319D10A500851040319272D282D512DAF
:101A5000D501D50A342D0130D035D10D890B2C2D6F
:101A60000130D4005408D507D11F372D382D2B2D28
:101A700051085302031D3E2D50085202031C412DF4
:101A8000422D462D5008D2025108D33B0130D136A9
:101A9000D00C890B472D0130D502031D502D512D3F
:101AA000382D56080319552D562D5B2DD209D30913
:101AB000D20A0319D30A5308D1005208D0000800F3
:101AC0002000D601D11F652D662D6D2DD009D109BD
:101AD000D00A0319D10AD601D60AD31F702D712D51
:101AE0007A2DD209D309D20A0319D30A0130D400BE
:101AF0005408D606D701D801500851040319812D86
:101B0000822DB12DD501D50A8E2D0130D035D10DC4
:101B1000890B862D0130D4005408D507D11F912D93
:101B2000922D852D0130D735D80D890B932D510875
:101B30005302031D9D2D50085202031CA02DA12D00
:101B4000A62D5008D2025108D33B57140130D1368C
:101B5000D00C890BA72D0130D502031DB02DB12D5E
:101B6000922D56080319B52DB62DBB2DD709D809CE
:101B7000D70A0319D80A5808D1005708D00008001E
:101B8000200049084A060319C62DC72DED2DD8306F
:101B9000D7009830D800953113258D3120003408B6
:101BA000003ED900F830353DDA00BA308F310427D5
:101BB0008D31BD30963163268D318E3127268D31A2
:101BC00020005D08B7005C08B6003708E60036085C
:101BD000E50097319E278D31262E0030D00004304D
:101BE000D1000030D2000C30D3003508D5003408C5
:101BF000D4008C3170248D3120005108B900500878
:101C0000B80039083506031D072E380834060319B5
:101C10000A2E0B2E262E3908B5003808B400D8300D
:101C2000D7009830D800953113258D312000340825
:101C3000003ED900F830353DDA00BA308F31042744
:101C40008D31BD30963163268D31DD2D0800173082
:101C5000963127268E31200051082100A700200050
:101C600050082100A6001730963127268E3120001B
:101C700050082100A607200051082100A73D0B3085
:101C80002000D0000030D100210027082000D30020
:101C9000210026082000D2008731DE278E31200067
:101CA00051082100A700200050082100A6002608A6
:101CB0002000A000210027082000A100A201A3010C
:101CC0003408D0003508D100890D893B8909D2003C
:101CD000D3002308D7002208D6002108D500200809
:101CE000D4008831F8208E3120005308A300520818
:101CF000A2005108A1005008A0000B30A336A20C8E
:101D0000A10CA00C890B7E2E21082100A700200029
:101D100020082100A60027082000DD002100260859
:101D20002000DC00080036302000D7009830D800B2
:101D3000953113258E312000C9013230D00000309A
:101D4000D1003308D3003208D2008A3118228E31F4
:101D5000200051082100B300200050082100B200EB
:101D60002000BE01BF0101302100A0070030A13DCD
:101D700022000C110E10D02E20003F082702031D58
:101D8000C32E3E0826020318C62EC72ECF2E2100D2
:101D9000B201B3012000CA01CA03C801C80A640025
:101DA000210032083304031DD62ED72EBC2E20006E
:101DB0004D08031DDC2EDD2EBC2E22000C150E144A
:101DC00021002F0820002502031DEA2E21002E08E5
:101DD00020002402031CED2EEE2EF22EFD30CA0050
:101DE000C801C80A210036080319F72EF82EFE2E66
:101DF00020002D08BD002C08BC00032F20002B085C
:101E0000BD002A08BC0008002000E400DA1F092FEA
:101E10000A2F122FD909DA09D90A0319DA0AE101BE
:101E2000E10A132FE1010730E3000A30D00000304F
:101E3000D1005A08D3005908D2008D310C258F31BA
:101E400020005008E2000A30D0000030D1005A08CB
:101E5000D3005908D2008D3160258F312000510800
:101E6000DA005008D900073063060319382F3A2FDB
:101E700001303B2F0030DB00DC015B086204DD0039
:101E80005C08DE0059085D04DF005A085E04E000CB
:101E90005F08600403194D2F4E2F582F6308640705
:101EA000DB005B08860087016208303E81006F2FEF
:101EB000610803195C2F5D2F672F63086407DB003F
:101EC0005B08860087012D308100E1016F2F6308D8
:101ED0006407DB005B088600870120308100FF304B
:101EE000DB005B08E307E31F762F772F152F6408CD
:101EF000083E860087018101080020003C083D045F
:101F00000319832F842FA32FFF30C400FF30C50097
:101F10004C0803198C2F8D2FFF2FCC01CF30D70009
:101F20009830D800953113258F3120003D08DA0014
:101F30003C08D900BA308F3104278F31BE3096313A
:101F400063268F31FF2F0130D8000030D9000330D5
:101F5000DA000030DB000230DC000030DD008331CD
:101F60008B238F3120005908B9005808B800380376
:101F70003904031DBC2FBD2FC02F2100A001A101DA
:101F800020008E1CC42FC52FCE2F3035C600310D3A
:101F9000C700FF30C400FF30C500F02F46084704DB
:101FA000031DD32FD42FF02FC51FD72FD82FE12FEC
:101FB0000D1FDB2FDC2FF02F2E35C4002F0DC50099
:101FC000F02F44084504031DE62FE72FF02F8E3134
:101FD00093268F31FF302000C400FF30C500F02F62
:101FE0004A084906031DF52FF62FFB2F4C0803194D
:101FF000FA2FFB2FFF2FCC01883160208F31080092
:1029200001340134013422008D168D1708008230E5
:102930002200970008001A30210097000800640068
:1029400080010131890BA02C0034013400340134A2
:1029500000340134013401346130320099009B01AC
:102960009D019F019E010800320091019201930197
:1029700094019501960108007C3020009E009D0185
:10298000911004309F000800833021009E009F01B9
:102990009B019C0101309D0008002000510821008E
:1029A000CF00200050082100CE00080080302C000D
:1029B0009900980197011F08FC3901389F00080011
:1029C00022008D1222008D1720008D1FE82CE92C8B
:1029D000E42C22008D16080022008D168D17200091
:1029E0008D1FF32CF42CEF2C22008D1222008D135E
:1029F00008002000D700D30101309631CD26943154
:102A00002000570896316326943108002000D70033
:102A1000D30100309631CD269531200057089631EC
:102A20006326953108002000D30100309631CD2671
:102A3000953120005808D4005708D3009531D82587
:102A4000953108002000D30101309631CD26953113
:102A500020005808D4005708D3009531D825953167
:102A60000800200051083100920020005008310079
:102A7000910015171514000000003100130808001C
:102A8000200090126F0896006E08950021004E08F5
:102A90004F0403194C2D4D2D522D4F088A004E081E
:102AA0000A00953108007708F9007608F800F93631
:102AB000F80CF936F80C78082C00980076080339E1
:102AC000F8000530F835FF3E031D622D783597007C
:102AD00008002000D2009431EC2495317C309731ED
:102AE0003E279531403097313E27953120005208DE
:102AF00097313E2795319431E0249531080020002C
:102B00006608DA006508D900BA308F31042795319C
:102B1000BD309431F9249531DC302000D300983059
:102B2000D4009531D8259531080020006608DA00D8
:102B30006508D900BA308F3104279531BB30943104
:102B4000F9249531E4302000D3009830D400953139
:102B5000D8259531080020006608DA006508D900FC
:102B6000BA308F3104279531BC309431F924953136
:102B700084302000D3009830D4009531D825953189
:102B80000800F3007308F200F20DF20D21001D0899
:102B90007206033972069D001D1421009D149D18B4
:102BA000D22DD32DCF2D1C08F1001B08F0000800FA
:102BB000E62D5308840054088500000895316925E6
:102BC000953101302000D3070030D43D2000530858
:102BD0008400540885001200031DEF2DF02DD92D1F
:102BE0000800403020009800E730960096309500AD
:102BF0001608EF001508EE00901221009016FE3026
:102C00002000D0000730D1009431CD249531903090
:102C10002000970008009431B42496319731CF27D3
:102C200096319431AC24963194319B249631943171
:102C3000972496319431C42496319431BC24963132
:102C40009431D62496319531F12596310800200033
:102C5000D3005308D200D20DD20D21001D08200050
:102C600052060339520621009D001D1421009D14B7
:102C70009D183B2E3C2E382E1C082000D100210030
:102C80001B082000D0000800F401F501701C492E3B
:102C90004A2E4E2E7208F4077308F53D0130F235C6
:102CA000F30D890B4F2E0130F136F00C890B542EA9
:102CB00070087104031D5D2E5E2E462E7508F1000E
:102CC0007408F00008002000D5005508D4007D2EBF
:102CD0005508860087010108953169259631013034
:102CE0002000D3005308D50754085502803A783E97
:102CF000031C7B2E7C2E7D2E852E55088600870199
:102D00000108031D842E852E682E08002000490826
:102D10004A0603198C2E8D2E942E7530D7009830CC
:102D2000D80095311325963120000E1F982E992E2C
:102D3000A12E8730D7009830D800953122259631C2
:102D4000A82EB430D7009830D8009531222596317E
:102D500008002000D2009431EC2496317C30973169
:102D60003E279631003097313E2796312000520899
:102D700097313E2796319431E02496312000520855
:102D8000FC390319C42EC52EC82E00320000CC2EEB
:102D90005330890BC92E000008002000D4000230F7
:102DA0009631A92696315330890BD42E000020008D
:102DB00054080319DC2EDD2EE52E5308C03ED50045
:102DC000003003180130D600EC2E5308803ED500A9
:102DD000003003180130D60055089631A9269631E7
:102DE000080000308B1B01302000D3005108310057
:102DF000920020005008310091002000520831005C
:102E00009300151715158B1355309600AA309600B0
:102E1000951495180C2F0D2F092F15112000530C08
:102E2000031C8B1303188B17080020005308D100D4
:102E30005208D0009531312597312000D400D501BA
:102E40005408D6005508D7000830D635D70D890B61
:102E5000252F5208013ED0000030533DD10095315E
:102E6000312597312000D400D5015408D6075508E4
:102E7000D73D5708D3005608D20008002000D000E4
:102E80008030D1005B2F22008D13200051085005A7
:102E900003194B2F4C2F4F2F22008D16512F22003C
:102EA0008D1203102000D10C22008D1720008D1FE1
:102EB0005A2F5B2F562F20005108031D602F612FC2
:102EC000432F22008D138D1622008D1720008D1F99
:102ED0006A2F6B2F662F22008D13080020004908EF
:102EE0004A06031D742F752F7A2F48080319792F6E
:102EF0007A2F8A2FC8011B30D7009830D80095311F
:102F00001325973120003F08E6003E08E5008B318D
:102F10005523973122000E100C11FA300032890B24
:102F20008E2F22000E140C15A1302000E700B530C2
:102F3000890B982FE70B982F0032080005302000EE
:102F4000E5070030E63D0A30D0000030D1006608C9
:102F5000D3006508D2008A31182297312000510829
:102F6000E6005008E5006608DA006508D900BA30C6
:102F70008F310427973121003E08BD003F08BE0075
:102F80002E30BF00BB309431F9249731E630200059
:102F9000D3009830D4009531D8259731080022000D
:102FA0008C01A0308D0001308E00333021008C0068
:102FB00050308D00CE308E00883023008E001030CF
:102FC0008D0030308C00A03024008D0003308C0048
:102FD00004308E0025008C018D018E0137302600D3
:102FE0008C00F0308D00FF308E003F3027008C00C9
:102FF000F0308D00FF308E0002303D00A50008004B
:103000002034203420342034203420342034203420
:10301000203457344134493454342034203420345B
:103020002034003454346534733474342034203400
:103030002034203400344F347634653472342034F4
:103040004134203420340034533465346E347334C6
:103050006F34723473342034003455347034203477
:10306000573461346934743420340034463449347C
:103070005234453420342134213421340034563440
:103080006F346C3474342034543468342E34003447
:1030900020342034203430342E3430343034413431
:1030A00000345434653473347434463469347234BF
:1030B0006534003450347234653473347334753489
:1030C0007234653400345734613474346534723486
:1030D00020345434683400344E346F342034573440
:1030E0006134743465347234003454346534733468
:1030F00074342034433464347334003453347034BF
:1031000072346134793420346D34733400342034B3
:10311000203420344E3469346734683474340034D5
:10312000443461347934203457346134693474342C
:1031300000344434613472346B345734613469344C
:103140007434003444346F3477346E34573461341B
:103150006934743400344C346F347734203456344A
:103160006F346C34743400342034203420342034F0
:103170002034443461347934003420347434693474
:103180006D346534733400342034203420343034CA
:1031900041340034543468342E34203400345734ED
:1031A000413449345434003441346B343D340034B8
:1031B00056346B343D340034733465346334003436
:1031C0004D346134783400342534003456340034BE
:020000040001F9
:08000000FF3FFF3FFF3FFF3F00
:08000E00EC3FFF3FFF3FFF3F05
:00000001FF
